:0200000480007A
:100000006F008004732F2034930F80006308FF0378
:10001000930F90006304FF03930FB0006300FF038E
:10002000130F000063040F0067000F00732F2034CC
:1000300063540F006F00400093E19153171F0000BD
:1000400023223FFC6FF09FFF732540F163100500F2
:10005000970200009382020173905230735000188F
:10006000970200009382020273905230B702008020
:100070009382F2FF7390023B9302F0017390023A75
:1000800097020000938282017390523073502030A7
:1000900073503030735040309301000097020000DD
:1000A000938282F673905230130510001315F501F8
:1000B000634C05000F00F00F930110009308D0056A
:1000C000130500007300000093020000638E02001D
:1000D00073905210B7B20000938292107390223046
:1000E00073232030E39A62F47350003097020000CB
:1000F0009382420173901234732540F173002030D3
:10010000370500809305008097260000938686EFD0
:1001100023A0A6002FA7B640B70E008093012000B1
:10012000631ED70383A70600930E0080930130005F
:100130006396D703930510002FA7B640930E008057
:1001400093014000631CD70183A70600930E108023
:10015000930150006394D701631030020F00F00F39
:10016000638001009391110093E111009308D00581
:1001700013850100730000000F00F00F93011000C1
:100180009308D0051305000073000000731000C031
:10019000000000000000000000000000000000005F
:1001A000000000000000000000000000000000004F
:0C01B00000000000000000000000000043
:1010000000000000000000000000000000000000E0
:1010100000000000000000000000000000000000D0
:1010200000000000000000000000000000000000C0
:1010300000000000000000000000000000000000B0
:081040000000000000000000A8
:040000058000000077
:00000001FF
